:100000000C942A000C9447000C9447000C94470071
:100010000C948E160C9447000C9447000C944700E7
:100020000C9447000C9447000C9447000C94470034
:100030000C9447000C9415170C9447000C9447003F
:100040000C9447000C9447000C9447000C94470014
:100050000C94470011241FBECFE5D8E0DEBFCDBF12
:1000600015E0A0E6B0E0E6E4FDE302C005900D92E5
:10007000A031B107D9F717E0A0E1B5E001C01D92AA
:10008000A73BB107E1F70E94E7020C94A11E0C9474
:100090000000EF92FF920F931F930E9433159398E5
:1000A00085E40E946815939A85E88A95F1F79398FC
:1000B00080E00E946815E82EFF2400E010E0102F79
:1000C0000F2DFE2CEE2480E00E94681590E0A0E049
:1000D000B0E0E82AF92A0A2B1B2B102F0F2DFE2C3B
:1000E000EE2480E00E946815939A282F30E040E0CB
:1000F00050E02E293F29402B512BB901CA011F91F5
:100100000F91FF90EF9008950E943315939881E02E
:100110000E946815939A939881E00E946815939ABB
:1001200008951F93182F0E943315939881E00E9421
:100130006815939A9398112311F082E001C083E02F
:100140000E946815939A1F9108951F930E9433157A
:100150009798979A939884E40E946815939A15E863
:10016000812F8A95F1F7939880E00E946815939A01
:10017000812F8A95F1F7939887E00E946815939AEA
:10018000812F8A95F1F7939883E00E946815939ADE
:10019000812F8A95F1F7939880E00E946815939AD1
:1001A000812F8A95F1F7939884E00E946815939ABD
:1001B000812F8A95F1F7939882E50E946815939AAA
:1001C000812F8A95F1F7939883E00E946815939A9E
:1001D000812F8A95F1F7939881E30E946815939A8D
:1001E000812F8A95F1F7939882E00E946815939A7F
:1001F000812F8A95F1F793988EE80E946815939A5B
:10020000812F8A95F1F7939881E00E946815939A5F
:10021000812F8A95F1F7939883E00E946815939A4D
:10022000812F8A95F1F7939884E40E946815939A38
:10023000812F8A95F1F7939880E00E946815939A30
:100240001A95F1F71F91089584B78093370514BE6E
:100250008898899A87B38C6087BBD798A798D698D7
:100260008AB38F638ABB84B38F6784BBBC9A81B324
:10027000886381BBC49A82B3886382BBBD9ABF9AEC
:10028000BE98C59AC79A8E988F9A8A9808952FB764
:100290008D5FF894A89591B5986191BD81BD2FBFF0
:1002A0000895582F6091480170914901482F4F5F80
:1002B000A82FAF5B342F3F73832F86958695869545
:1002C000FB01E80FF11D808190E0232F277002C011
:1002D000959587952A95E2F780FD04C04F5F4A17F0
:1002E00049F7352F832F089581E08093120560919F
:1002F000540170915501409156015091570120E0F1
:1003000030E0FB01E20FF31FDA01A20FB31F90816F
:100310008C91981719F01092120505C02F5F3F4F6E
:100320002B30310571F781E0809310056091480111
:100330007091490140914A0150914B0120E030E019
:10034000FB01E20FF31FDA01A20FB31F90818C9122
:10035000981719F01092100508952F5F3F4F28301D
:10036000310571F7089581E080931205609156017F
:1003700070915701409154015091550120E030E0B7
:10038000FB01E20FF31F80818095FA01E20FF31F5A
:100390009081892319F01092120505C02F5F3F4FFD
:1003A0002B30310569F780911205089581E0809323
:1003B000100560914A0170914B01409148015091A4
:1003C000490120E030E0FB01E20FF31F80818095BE
:1003D000FA01E20FF31F9081892319F010921005A2
:1003E00005C02F5F3F4F2830310569F78091100518
:1003F0000895CF92DF92EF92FF920F931F93CF93C6
:10040000DF93E82EC0905401D0905501C0E0D0E0B9
:10041000082F10E00F5F1F4FC8018C0F9D1F64E570
:1004200070E00E94351EF82E869586958695F60119
:10043000E80FF11D808190E02F2D277002C0959567
:1004400087952A95E2F780FF0BC0809114058823D9
:10045000B1F08F2D63E00E9495170E94DB160FC04C
:100460002196C435D105C1F680911405882331F059
:100470008E2D63E00E9495170E94DB16FE2C8F2DB7
:10048000DF91CF911F910F91FF90EF90DF90CF9070
:10049000089580E690E00E94E416089588EA90E0CE
:1004A0000E94E41680919107853020F19091940785
:1004B000892F81548830F0F4892F0E94D7168AEC56
:1004C00090E00E94E416809196070E948B178AE0C4
:1004D0000E94D71680919407E0914801F09149015C
:1004E000E80FF11DE154F0408091960780838091E0
:1004F000940732C083E08093910790919307892FEE
:100500008154883098F5892F0E94D71680919407DE
:10051000803389F08FEC90E00E94E416809193077D
:10052000E0914801F0914901E80FF11DE154F040DC
:100530008FEF80830FC089ED90E00E94E4168091D8
:100540009307E0914801F0914901E80FF11DE15452
:10055000F040108280919307E0914A01F0914B01A5
:10056000E80FF11DE154F0401082089583EE90E011
:100570000E94E41686EF90E00E94E41680919107B5
:1005800063E00E9495178EE091E00E94E41680914E
:1005900094070E94D71685E291E00E94E4168091AC
:1005A00096070E948B178AE00E94D716089586B19D
:1005B000866086B93098359A80B78F7180BF379A38
:1005C0003E983F9887B1866087B9369A0895CF9252
:1005D000DF92EF92FF920F931F93CF93DF930E94CE
:1005E00024010E94CA160E9427150E9483160E94A9
:1005F000D7020E943F050E94BB070E94A500789485
:1006000080E090E02FEFE0914801F0914901E80F80
:10061000F91F2083E0914A01F0914B01E80FF91F87
:10062000108201968830910571F780E090E03FE0FC
:100630002FEFE0915401F09155018A3021F0E80F3D
:10064000F91F208301C03287E0915601F0915701D4
:10065000E80FF91F108201968B30910551F786EA59
:1006600091E00E94E4160E94DB1660E2C62E6EE462
:10067000D62E0E944508082F873159F0843149F061
:100680008EE591E00E94E416802F0E948B170E9455
:10069000DB1680912B0590912C0569E170E00E949A
:1006A000211E892B11F5809116058823F1F00E94F7
:1006B0007705EC010097C9F00E947705C817D907A4
:1006C00021F00E947705EC01F7CF85E791E00E94C9
:1006D000E416CE0167E00E9481170E94DB1684E0D9
:1006E00061E00E94FA050E9402120E94B301882371
:1006F00089F1809113058823F1F08DE791E00E9444
:10070000E41660912D0570912E0580912F05909132
:10071000300548E00E94721780E090E061E070E0F0
:100720000E94430E0E9470100E9404100E9412103A
:100730000E9404100FC08091A401882359F481E025
:100740008093A40181E090E061E070E00E94430E9C
:100750000E9470100E94D601882301F1809111053A
:10076000882359F00E94EE0E0E9470100E94E30F41
:100770000E9404100E94121011C08091A3018823CE
:1007800069F481E08093A30181E090E061E070E092
:100790000E94EE0E0E9470100E94E30F80912507C8
:1007A000882321F08BB398E089278BBB909131058A
:1007B000992381F05D9B0EC08091B2078CB9E2EB6A
:1007C000F7E08181819387E0E73BF807D1F791500B
:1007D000909331055B9B05C080E891E00E94E41690
:1007E0008CB180913305882311F00E948A12349BCA
:1007F000B9C080911205882309F0B4C094B185B1C5
:10080000349AE0915C01F0915D01F82EEE24292FDD
:1008100030E02E293F2931832083809114058823DD
:1008200029F0C9010E9477170E94DB16E091580158
:10083000F09159018081C0915C01D0915D01A0913E
:100840005A01B0915B0120915201309153018832DD
:1008500009F03EC0EC91F0E0EE0FFF1FE20FF31F36
:100860008081918128813981820F931F91838083B8
:100870002C91822F869586958695E0915601F09170
:100880005701E80FF11D277081E090E002C0880F4A
:10089000991F2A95E2F72081282B208300915A0185
:1008A00010915B01F80180810E94F901F8018083B9
:1008B000E0915A01F0915B0180810E946F08E09104
:1008C0005801F09159011082C6010197F1F74AC011
:1008D000EC91F0E0EE0FFF1FE20FF31F808191819A
:1008E00028813981820F931F918380838091140521
:1008F000882389F185E991E00E94E416E0915A018C
:10090000F0915B01808164E00E94951789E991E094
:100910000E94E416E0915C01F0915D01808191817B
:100920000E9477178DE991E00E94E416E0915A0148
:10093000F0915B01808190E0880F991FE091520156
:10094000F0915301E80FF91F8081918168E00E94C6
:1009500081170E94DB16E0915801F09159018081C6
:100960008F5F8083869985CE80911005882309F05A
:1009700080CE00915001109151010E944900F80170
:100980006083718382839383C0914C01D0914D0128
:100990008881823009F05EC0E0914E01F0914F01F4
:1009A000808190E0880F991F880F991FE091460180
:1009B000F0914701E80FF91FA0915001B09151014A
:1009C0008D919D910D90BC91A02D80839183A283E8
:1009D000B383188280911405882381F0E09150013F
:1009E000F091510160817181828193810E94681729
:1009F0008AE00E94D7168AE00E94D716E0914E0145
:100A0000F0914F012081822F869586958695E09101
:100A10004A01F0914B01E80FF11D277081E090E051
:100A200002C0880F991F2A95E2F72081282B208386
:100A300000914E0110914F01F80180810E945101F7
:100A4000F8018083E0914E01F0914F0180810E9476
:100A5000A3080FCE8F5F888380911405882309F443
:100A600008CEE0915001F091510160817181828145
:100A700093810E9468178AE00E94D716FACDC29827
:100A800084EF91E028EC30E0F9013197F1F701971C
:100A9000D9F7C29A80E197E20197F1F708950F9391
:100AA0001F938C010E9440158FE080936E07109376
:100AB0006F07009370071092710784E00E946A1616
:100AC000809184071F910F9108950F931F9388E2DF
:100AD00094E00E944F05182F00E089E294E00E9404
:100AE0004F05080F111DC8011F910F9108951F9305
:100AF00086E294E00E944F05182F87E294E00E945E
:100B00004F05512F40E0282F30E0242B352BC90111
:100B10001F9108950F931F9384E294E00E944F0564
:100B2000182F00E085E294E00E944F05080F111D88
:100B3000C8011F910F9108950F931F9382E294E0D3
:100B40000E944F05182F00E083E294E00E944F05B9
:100B5000080F111DC8011F910F9108950F931F9346
:100B600080E294E00E944F05182F00E081E294E0BB
:100B70000E944F05080F111DC8011F910F91089584
:100B800083E094E00E944F05089583E094E00E9482
:100B90004F05873121F481E08093150502C0109242
:100BA0001505809115050895FF920F931F93F82E58
:100BB000192F062F0E94401580EF80936E07109327
:100BC0006F07F09270070093710784E00E946A1625
:100BD0001F910F91FF9008951F93182F692F88E29E
:100BE00094E00E94D40589E294E0612F0E94D4052C
:100BF0001F9108954F925F926F927F929F92AF9252
:100C0000BF92CF92DF92EF92FF920F931F93CF93F9
:100C1000DF93082F0E9477059C01009711F4992417
:100C200089C0902E84E0801710F444E0942E892D22
:100C300090E02817390708F4922E0E9465053C01C0
:100C4000EC01DF70C12C90E6D92ECC0EDD1E83ECBA
:100C500091E00E94E416C3010E9477170E94DB1600
:100C600088EC91E00E94E416CE010E9477170E9462
:100C7000DB168DEC91E00E94E416C6010E94771706
:100C80000E94DB16A92CBB24C5018C0F9D1F81502F
:100C9000904118F4C0E0D0E037C0E12C80E1F82E9C
:100CA000EC1AFD0A25014E185F0800E009C0CE01CC
:100CB0008C0D9D1D0E944F05C95DD84F88830F5F25
:100CC000C02FD0E0CE15DF0590F3DD240CC08C01E1
:100CD0000E0D1F1D8050904A0E944F05095D184F50
:100CE000F8018083D3948D2D90E08415950578F3D9
:100CF0000DC0C6010E944F05FE01E95DF84F8083DB
:100D000021960894C11CD11CC91598F38501060DC4
:100D1000171D82ED91E00E94E416C8010E9477172A
:100D20000E94DB16C8010E94EC0581E094E060E4BB
:100D30000E94D405892DDF91CF911F910F91FF90D3
:100D4000EF90DF90CF90BF90AF909F907F906F908B
:100D50005F904F9008951F93182F692F84E294E0BD
:100D60000E94D40585E294E0612F0E94D4051F9172
:100D700008956F927F928F929F92AF92BF92CF927F
:100D8000DF92EF92FF920F931F93CF93DF933C017B
:100D90006B010E94AE055C0110E00E94AE05A81632
:100DA000B90621F00E94AE055C0101C01F5F13303F
:100DB000A0F3A114B10419F4CC24DD2474C00E9462
:100DC0008A054C0110E00E948A058816990621F0D8
:100DD0000E948A054C0101C01F5F1330A0F3E4019B
:100DE000DF70E12C50E4F52EEC0EFD1E809117050E
:100DF000909118058815990521F087ED91E00E94E2
:100E0000E416AC14BD0408F46501C6018C0F9D1FE7
:100E10008150904118F4C0E0D0E034C000E010E10F
:100E20000C1B1D0B5601A01AB10AC0E0D0E0F30163
:100E3000EC0FFD1FC70160810E94D4052196089424
:100E4000E11CF11CC017D10790F3060D171DC0E07F
:100E5000D0E009C0CE018050904AF80161918F0125
:100E60000E94D4052196CA15DB05A0F30EC0F3013C
:100E7000EC0FFD1FC70160810E94D40521960894E4
:100E8000E11CF11CCC15DD0590F3C601880D991D00
:100E900090931805809317050E94AB0681E094E0BB
:100EA00060E20E94D405C601DF91CF911F910F919E
:100EB000FF90EF90DF90CF90BF90AF909F908F907A
:100EC0007F906F90089590912607903248F4E92F13
:100ED000F0E0E45DF84F8AE080839F5F90932607FF
:100EE000609126078CE297E070E00E94B9061092AC
:100EF00026070895DC010BC09032F0F7E92FF0E0EF
:100F0000E45DF84F80839F5F9093260711968C9144
:100F100090912607882381F7903248F4E92FF0E07A
:100F2000E45DF84F8AE080839F5F9093260760918D
:100F300026078CE297E070E00E94B906109226071F
:100F40000895DC010BC06032F0F7E62FF0E0E45DBD
:100F5000F84F80836F5F6093260711968C916091A4
:100F60002607882381F78CE297E070E00E94B9069B
:100F700010922607089589E090E06AEF0E94D40558
:100F80008AE090E067EC0E94D4058BE090E06FE08F
:100F90000E94D4058CE090E06DEA0E94D4058DE0BB
:100FA00090E062E20E94D4058EE090E061E00E9451
:100FB000D4058FE090E06AE00E94D40580E190E0E3
:100FC00060E00E94D40581E190E060E80E94D405D1
:100FD00082E190E06FE70E94D40585E090E06FEF3A
:100FE0000E94D40586E090E06FEF0E94D40587E070
:100FF00090E06FEF0E94D40588E090E060E00E94EE
:10100000D40581E090E06AE00E94D40582E090E09F
:1010100060E00E94D40583E090E060E00E94D40587
:1010200084E090E060E00E94D4058AE190E06AE00C
:101030000E94D4058BE190E06AE00E94D40580E034
:1010400094E061E00E94D40584E094E063E10E94B2
:10105000D40585E094E068E80E94D40581E094E03E
:1010600061E00E94D40583E094E00E944F05833143
:10107000D1F781E094E062E00E94D40583E094E03F
:101080000E944F058431D1F708951F930E94C00537
:10109000182F80912B07181729F0812F0E948B178A
:1010A0000E94DB1610932B07173139F0143159F0D9
:1010B0000E94C005182F873121F481E08093160526
:1010C0000BC0843119F41092160506C01092160553
:1010D0000E943F050E94BB07812F1F91089588320F
:1010E00048F4282F30E0843210F02F5F3F4F922FCA
:1010F000990F23C0803560F48852282F30E0843265
:1011000010F02F5F3F4F220F331F922F9F5F15C0AC
:10111000843590F48055813049F0813028F0823058
:1011200039F0833049F406C098E407C099E405C05B
:1011300092E503C093E501C090E085B39F77807886
:10114000982B95BB0895282F82958F70823041F09F
:10115000833041F0882311F490E105C090E003C092
:1011600090E301C090E28BB32F70922B807C982B80
:101170009BBB0895982F92959F70ADEEB1E0FD0155
:10118000E90FF11D908190934C078F70A80FB11D4E
:101190008C9180934D0710924E078CE497E0089550
:1011A000ECE4F7E027E0482F50E060E331E3CA01C8
:1011B000022E02C0959587950A94E2F7DF011196F9
:1011C00080FF02C0308301C06083FD01215078F7A9
:1011D0001C928CE497E00895292F22952F70ADEE94
:1011E000B1E0FD01E20FF11D208120934C079F70BB
:1011F000FD01E90FF11D908190934D07982F929575
:101200009F70FD01E90FF11D908190934E078F7043
:10121000A80FB11D8C9180934F07109250078CE45A
:1012200097E00895292F22952F70ADEEB1E0FD01D2
:10123000E20FF11D208120934C079F70FD01E90F03
:10124000F11D908190934D07982F92959F70FD010D
:10125000E90FF11D908190934E078F70FD01E80F0B
:10126000F11D808180934F07872F82958F70FD013C
:10127000E80FF11D8081809350077F70FD01E70F1B
:10128000F11D808180935107862F82958F70FD011B
:10129000E80FF11D8081809352076F70A60FB11D7A
:1012A0008C9180935307109254078CE497E0089533
:1012B000CF93DF93EC01FC0101900020E9F7319717
:1012C000E81BACE5B7E080E202C08D936150E61701
:1012D000E0F3CD018E0F911DFC0102C089918D9329
:1012E000AE17BF07D9F71C928CE597E0DF91CF913D
:1012F00008952F923F924F925F926F927F928F92BA
:101300009F92AF92BF92CF92DF92EF92FF920F9394
:101310001F93DF93CF930F92CDB7DEB75B016C01C4
:101320002983242E85E0841710F435E0232EC6018E
:10133000B501A60195010E94CA1A882359F08EE6CC
:1013400080934E0780934C0781E680934D0710925F
:101350004F07BBC0C601B50120E030E040E050E0DF
:101360000E949A1A87FD05C02CE4422E27E0522ED7
:101370000BC08DE280934C07D7FAD094D7F8D09465
:101380009DE4492E97E0592EC601B5010E949A1797
:101390003B014C01611571058105910521F480E344
:1013A000D2018D932D0184017301332423C0C80120
:1013B000B7012AE030E040E050E00E94481EE32DF3
:1013C000F0E0E75EFA4F6083E61AF10801091109BF
:1013D000E114F1040105110561F0C801B7012AE02B
:1013E00030E040E050E00E94481EC901DA017C0173
:1013F0008D013394E114F10401051105C1F6C40116
:10140000B3010E94A71B9B01AC01C601B5010E945C
:1014100012197B018C0181E2A82E85E0B82E6501AE
:10142000822C99243501680C791C22C0C801B701AF
:1014300020E030E040E251E40E9470197B018C0111
:101440000E949A17F6016083662379F070E088277E
:1014500077FD8095982F0E94F51A9B01AC01C80179
:10146000B7010E9412197B018C010894C11CD11C88
:10147000C614D704D9F6932D9150A92FBB27A7FDE9
:10148000B095A75EBA4F07C08C91805DF201808352
:1014900029019150119792012F5F3F4F97FFF4CF91
:1014A0008EE2D2018C93F20105C0D5018D915D01D0
:1014B000805D80833196AC14BD04B9F7280D391DC9
:1014C000F9011082F981FF2319F42CE437E006C0FA
:1014D0008CE497E069810E9458099C01C9010F9032
:1014E000CF91DF911F910F91FF90EF90DF90CF9000
:1014F000BF90AF909F908F907F906F905F904F9034
:101500003F902F900895BF92CF92DF92EF92FF927B
:101510000F931F93CF93DF938B019C01B42E97FF02
:101520000DC08DE280934C07CC24DD247601C01AD7
:10153000D10AE20AF30ACDE4D7E004C06B017C01D2
:10154000CCE4D7E080E0C8168AECD8068AE9E80641
:101550008BE3F80658F0C701B60120E03AEC4AE9FF
:101560005BE30E94481E205D299309C080E0C816F5
:1015700081EED80685EFE80685E0F80688F0C70119
:10158000B60120E03AEC4AE95BE30E94481E20E005
:1015900031EE45EF55E00E94481E205D299309C0B9
:1015A00080E8C81686E9D80688E9E80680E0F806EB
:1015B00088F0C701B60120E031EE45EF55E00E940A
:1015C000481E20E836E948E950E00E94481E205DA8
:1015D000299309C080E4C81682E4D8068FE0E806A3
:1015E00080E0F80688F0C701B60120E836E948E94E
:1015F00050E00E94481E20E432E44FE050E00E9498
:10160000481E205D299309C080EAC81686E8D806DE
:1016100081E0E80680E0F80688F0C701B60120E422
:1016200032E44FE050E00E94481E20EA36E841E0F4
:1016300050E00E94481E205D299309C080E1C81631
:1016400087E2D80680E0E80680E0F80688F0C70167
:10165000B60120EA36E841E050E00E94481E20E151
:1016600037E240E050E00E94481E205D299309C007
:1016700088EEC81683E0D80680E0E80680E0F80629
:1016800088F0C701B60120E137E240E050E00E9457
:10169000481E28EE33E040E050E00E94481E205DE6
:1016A000299306C084E6C816D104E104F10488F049
:1016B000C701B60128EE33E040E050E00E94481E2A
:1016C00024E630E040E050E00E94481E205D29936F
:1016D00006C08AE0C816D104E104F10480F0C70115
:1016E000B60124E630E040E050E00E94481E2AE0C7
:1016F00030E040E050E00E94481E205D2993C70181
:10170000B6012AE030E040E050E00E94481E605DF3
:1017100068831982BB2019F42CE437E006C08CE4FE
:1017200097E06B2D0E9458099C01C901DF91CF9170
:101730001F910F91FF90EF90DF90CF90BF90089591
:10174000DF92EF92FF920F931F93CF93DF937B0172
:101750008C01D42E80E0E8168AECF8068AE90807A6
:101760008BE3180770F0C801B70120E03AEC4AE9B2
:101770005BE30E94481E205D20934C07CDE4D7E038
:101780000BC080E0E81681EEF80685EF080785E0DB
:10179000180798F0CCE4D7E0C801B70120E03AEC94
:1017A0004AE95BE30E94481E20E031EE45EF55E038
:1017B0000E94481E205D29930BC080E8E81686E948
:1017C000F80688E9080780E0180798F0CCE4D7E02D
:1017D000C801B70120E031EE45EF55E00E94481EF8
:1017E00020E836E948E950E00E94481E205D299330
:1017F0000BC080E4E81682E4F8068FE0080780E07A
:10180000180798F0CCE4D7E0C801B70120E836E922
:1018100048E950E00E94481E20E432E44FE050E0E6
:101820000E94481E205D29930BC080EAE81686E8D6
:10183000F80681E0080780E0180798F0CCE4D7E0CC
:10184000C801B70120E432E44FE050E00E94481E96
:1018500020EA36E841E050E00E94481E205D2993CE
:101860000BC080E1E81687E2F80680E0080780E018
:10187000180798F0CCE4D7E0C801B70120EA36E8B1
:1018800041E050E00E94481E20E137E240E050E095
:101890000E94481E205D29930BC088EEE81683E065
:1018A000F80680E0080780E0180798F0CCE4D7E05D
:1018B000C801B70120E137E240E050E00E94481E35
:1018C00028EE33E040E050E00E94481E205D29935E
:1018D00008C084E6E816F1040105110598F0CCE48F
:1018E000D7E0C801B70128EE33E040E050E00E94A5
:1018F000481E24E630E040E050E00E94481E205D93
:1019000029930BC08AE0E816F1040105110518F4CB
:10191000CCE4D7E012C0CCE4D7E0C801B70124E69C
:1019200030E040E050E00E94481E2AE030E040E015
:1019300050E00E94481E205D2993C801B7012AE0AB
:1019400030E040E050E00E94481E605D68831982EC
:10195000DD2019F42CE437E006C08CE497E06D2D0F
:101960000E9458099C01C901DF91CF911F910F91ED
:10197000FF90EF90DF900895CF93DF939C01462F67
:1019800097FF0AC08DE280934C07EE27FF27E21BEA
:10199000F30BCDE4D7E003C0FC01CCE4D7E087E251
:1019A000E031F80740F0CF0160E177E20E94211EAC
:1019B000605D699304C083E0E83EF80760F0CF0102
:1019C00060E177E20E94211E68EE73E00E94211E12
:1019D000605D699303C0E436F10560F0CF0168EE05
:1019E00073E00E94211E64E670E00E94211E605D8B
:1019F000699303C0EA30F10558F0CF0164E670E066
:101A00000E94211E6AE070E00E94211E605D6993C1
:101A1000CF016AE070E00E94211E805D88831982F8
:101A2000442319F42CE437E006C08CE497E0642FDB
:101A30000E9458099C01C901DF91CF9108959C0132
:101A4000462F87E22031380758F0C90160E177E27C
:101A50000E94211E605D60934C07EDE4F7E006C034
:101A600083E0283E380770F0ECE4F7E0C90160E15C
:101A700077E20E94211E68EE73E00E94211E605DE5
:101A8000619305C02436310570F0ECE4F7E0C9013C
:101A900068EE73E00E94211E64E670E00E94211E41
:101AA000605D619308C02A30310518F4ECE4F7E07A
:101AB0000DC0ECE4F7E0C90164E670E00E94211E6D
:101AC0006AE070E00E94211E605D6193C9016AE0D6
:101AD00070E00E94211E805D80831182442319F4EE
:101AE0002CE437E006C08CE497E0642F0E9458098C
:101AF0009C01C9010895982F362F87FF08C08DE2F9
:101B000080934C07292F2195EDE4F7E003C0282F9F
:101B1000ECE4F7E0243668F0822F90E068EE73E0A2
:101B20000E94351E64E670E00E94351E605D619380
:101B300002C02A3050F0822F64E60E94151E892FC1
:101B40006AE00E94151E805D8193822F6AE00E94E8
:101B5000151E905D90831182332319F42CE437E035
:101B600006C08CE497E0632F0E9458099C01C901CC
:101B700008951F93482F162F843678F090E068EE72
:101B800073E00E94351E64E670E00E94351E605DC1
:101B900060934C072DE437E007C08A3018F4ECE47A
:101BA000F7E00DC02CE437E0842F64E60E94151E98
:101BB000892F6AE00E94151E805DF9018193842FB0
:101BC0006AE00E94151E905D90831182112319F422
:101BD0002CE437E006C08CE497E0612F0E9458099E
:101BE0009C01C9011F9108958EEF91E00E94E416B7
:101BF00008951F93CF93DF93182FEB01803508F5DD
:101C000068E20E94151E96959695963028F49430B9
:101C100070F4923040F009C0983069F0983048F084
:101C2000993069F40AC081E40DC082E40BC083E4FA
:101C300009C084E407C085E405C086E403C08FE3DF
:101C400001C088E40E94D716812F68E20E94151E09
:101C50009452943010F4137001C01770812F8F5F6D
:101C600061E00E9495178AE30E94D716CE016AE0D0
:101C700070E00E94211ECB0167E00E948117DF9176
:101C8000CF911F9108951F93CF93DF9389E192E045
:101C90000E94E416C0E0D0E01C2FCE018770907047
:101CA000892B19F48AE00E94D716CE01880F991F5C
:101CB000E0915201F0915301E80FF91F60817181A9
:101CC000812F0E94F90D85E392E00E94E41621968F
:101CD000C435D10509F78AE00E94D716DF91CF916C
:101CE0001F9108951F93CF93DF9389E392E00E94A1
:101CF000E41610E0C0E0D0E081E692E00E94E41635
:101D0000812F63E00E94951780E20E94D716E09130
:101D10005201F0915301EC0FFD1F808191810E94CF
:101D2000771780E20E94D716E0915201F09153019B
:101D3000EC0FFD1F8081918167E00E9481170E9456
:101D4000DB161F5F22961435B9F68AE00E94D7167B
:101D5000DF91CF911F91089580E480932C078093A9
:101D60002D078CE297E062E070E00E94B9060895CA
:101D7000CF92DF92EF92FF921F93182F6A017B019F
:101D800085E692E00E94E416812F869586958695D9
:101D90008F5B0E94D7161770812F8F5F61E00E94C2
:101DA00095178AE30E94D716C701B6010E94A71BA8
:101DB00020E030E048EC50E40E94701920E030E070
:101DC00040E053E30E94701943E026E00E9463174D
:101DD0001F91FF90EF90DF90CF900895CF92DF9208
:101DE000EF92FF920F931F93CF93DF9388E692E0D9
:101DF0000E94E416C0E0D0E0EE24FF240C2F37E070
:101E0000C32ED12CCC22DD22C114D10419F48AE0D6
:101E10000E94D71685E692E00E94E416102F1695D0
:101E200016951695812F8F5B0E94D7160770802F0D
:101E30008F5F61E00E9495178AE30E94D716E091B8
:101E40004801F0914901E10FF11D808190E002C04D
:101E500095958795CA94E2F780FF1FC0E0914601EF
:101E6000F0914701EE0DFF1D6081718182819381A8
:101E70000E94A71B2DEC3CEC4CEC50E40E94701926
:101E800020E030E040E053E30E94701943E026E098
:101E90000E94631782E992E002C084E992E00E9406
:101EA000E416219684E090E0E80EF91EC034D105D6
:101EB00009F0A4CFDF91CF911F910F91FF90EF9088
:101EC000DF90CF9008950E94430E0E94EE0E089579
:101ED000CF93DF938CE992E00E94E416C0E0D0E05B
:101EE000E0915401F0915501EC0FFD1F80810E949B
:101EF000861780E20E94D7162196CB30D10581F754
:101F00000E94DB16C0E0D0E0E0915601F09157014D
:101F1000EC0FFD1F80810E94861780E20E94D71679
:101F20002196CB30D10581F70E94DB1689EA92E039
:101F30000E94E416C0E0D0E0E0914801F091490130
:101F4000EC0FFD1F80810E94861780E20E94D71649
:101F50002196C830D10581F70E94DB16C0E0D0E0A1
:101F6000E0914A01F0914B01EC0FFD1F80810E942E
:101F7000861780E20E94D7162196C830D10581F7D6
:101F80000E94DB1689EB92E00E94E41660912D0519
:101F900070912E0580912F05909130054AE00E94A6
:101FA00072178FEB92E00E94E416DF91CF910895B3
:101FB00008958091290790912A07E8E3F5E0E80F5A
:101FC000F11D9083089580E090E0E0914A01F09146
:101FD0004B01E80FF91F1082019688309105A9F78F
:101FE0000895209146013091470180E090E0F90189
:101FF000E80FF91F1082118212821382049641E0C9
:1020000080309407A1F7089580E090E0E0915601B8
:10201000F0915701E80FF91F108201968B3091055E
:10202000A9F70895209152013091530180E090E08A
:10203000F901E80FF91F118210820296883A910582
:10204000B9F7089580E090E0E0914A01F0914B01EA
:10205000E80FF91F1082019688309105A9F780E0FA
:1020600090E0E0915601F0915701E80FF91F1082BE
:1020700001968B309105A9F70895EF92FF921F9377
:10208000DF93CF93CDB7DEB72D970FB6F894DEBFB1
:102090000FBECDBFDE011196E6ECF2E08DE00190BF
:1020A0000D928150E1F710E07E010894E11CF11CD3
:1020B000812F64E00E94B90D0E94A107C7010E9410
:1020C000A1071F5F1F3FA1F72D960FB6F894DEBF43
:1020D0000FBECDBFCF91DF911F91FF90EF9008957C
:1020E000EF92FF920F931F93CF93DF9383ED92E0D4
:1020F0000E94A10760913C0170913D01882777FD06
:102100008095982F0E9412090E947A07F8948CED0E
:1021100092E00E94A10760912D0570912E0580919B
:102120002F059091300541E00E94A00B0E94A1076D
:1021300085EE92E00E94A10780912B0590912C05DD
:1021400061E00E941F0D0E947A07789487EE92E06A
:102150000E947A0781EF92E00E94A107C0E0D0E0E0
:1021600010E2E0915401F0915501EC0FFD1F8081C8
:102170000E94D0080E94A10780912607E82FF0E076
:10218000E45DF84F1083982F9F5F90932607219668
:10219000CB30D10531F7E92FF0E0E45DF84F8AE06C
:1021A00080839F5F9093260789EF92E00E94A107AA
:1021B000C0E0D0E010E2E0915601F0915701EC0F41
:1021C000FD1F80810E94D0080E94A10780912607F0
:1021D000E82FF0E0E45DF84F1083982F9F5F909315
:1021E00026072196CB30D10531F7E92FF0E0E45DE9
:1021F000F84F8AE080839F5F9093260781E093E009
:102200000E94A107C0E0D0E010E2E0915201F091FD
:102210005301EC0FFD1F808191816AE070E00E9404
:10222000211ECB0161E00E941F0D0E94A107809139
:102230002607E82FF0E0E45DF84F1083982F9F5FAA
:10224000909326072296C83AD105F9F6E92FF0E0D7
:10225000E45DF84F8AE080839F5F9093260789E0D2
:1022600093E00E947A0781EF92E00E94A107C0E00C
:10227000D0E010E2E0914801F0914901EC0FFD1F20
:1022800080810E94D0080E94A10780912607E82F34
:10229000F0E0E45DF84F1083982F9F5F909326073E
:1022A0002196C830D10531F7E92FF0E0E45DF84F11
:1022B0008AE080839F5F9093260789EF92E00E94D7
:1022C000A107C0E0D0E010E2E0914A01F0914B019B
:1022D000EC0FFD1F80810E94D0080E94A107809111
:1022E0002607E82FF0E0E45DF84F1083982F9F5FFA
:1022F000909326072196C830D10531F7E92FF0E0F9
:10230000E45DF84F8AE080839F5F9093260786E123
:1023100093E00E94A107C0E0D0E000E010E090E26E
:10232000E92E8AE0F82EE0914601F0914701E00F96
:10233000F11F60817181828193810E94A71B20E03F
:1023400030E048EC55E40E94701920E030E040E0B5
:1023500053E30E94701942E022E00E9479090E9432
:10236000A107CE0187709070E0912607079729F4A6
:10237000F0E0E45DF84FF08204C0F0E0E45DF84F77
:10238000E082809126078F5F8093260721960C5F5D
:102390001F4FC034D10539F68FE193E00E947A07D0
:1023A000DF91CF911F910F91FF90EF900895809151
:1023B000270780932C078091280780932D078CE2B4
:1023C00097E062E070E00E94B906089580912707C7
:1023D00080932C078091280780932D0780912907EF
:1023E00080932E0780912907E8E3F5E0E80FF11DBF
:1023F000808180932F078CE297E064E070E00E9478
:10240000B9060895FF920F931F93CF93DF93F82E91
:1024100086E293E00E940A17C0E0D0E08E01095DD9
:10242000184FF80180810E948B17F80180810E946B
:10243000D7162196C430D10589F70E94DB16FF20FC
:1024400009F462C080912707833709F44CC08437B0
:1024500048F48D3609F441C08237D1F08B3609F04B
:1024600053C044C0863739F1873720F4843709F0E8
:102470004BC011C0873721F08A3709F045C039C0F9
:10248000E091290780912A07F0E0E85CFA4F808309
:102490000E94E61139C01092A30180E090E0E09123
:1024A0004A01F0914B01E80FF91F10820196883024
:1024B0009105A9F70FC01092A40180E090E0E0918F
:1024C0005601F0915701E80FF91F108201968B30E9
:1024D0009105A9F70E94D71117C00E94221081E030
:1024E0008093110511C00E9470100EC00E943D1013
:1024F0000BC081E280932C0780932D078CE297E03C
:1025000062E070E00E94B906DF91CF911F910F91B8
:10251000FF9008950F931F931092B10780E20E94DD
:10252000D71682E997E00E94E4168AE00E94D71647
:1025300090919107992309F4B8C08091920782364F
:1025400009F44CC18336B8F4873409F456C1883491
:1025500040F4843439F1853419F1813209F0A5C091
:102560008CC1803509F478C1833509F483C188347E
:1025700009F09BC097C1873609F451C1883630F401
:10258000843681F0853609F090C00AC0803709F49E
:1025900058C1833709F46BC1883609F086C082C1FF
:1025A00001E001C000E080919307823739F086375F
:1025B00029F0883619F0803709F077C0933010F48D
:1025C00010E006C01091940710531A3008F06DC047
:1025D000943058F09091950790539A3048F48AE0DF
:1025E000189F102D1124190F03C0933008F45DC0FB
:1025F0008FE293E00E94E416002319F080E493E058
:1026000002C084E493E00E94E4168091930780372F
:1026100009F4B1C0813720F4883609F0DCC07FC0EE
:10262000823721F0863709F0D6C042C0412F469547
:1026300046954695E0914801F0914901612F70E07F
:10264000002379F0E40FF11D6770707081E090E075
:1026500002C0880F991F6A95E2F72081282B2083FA
:1026600019C050E0E40FF51F6770707021E030E092
:1026700002C0220F331F6A95E2F7209580818223E2
:102680008083E0914A01F0914B01E40FF51F8081B6
:102690008223808389E493E00E94E416812F62E024
:1026A0000E9495178AE00E94D716E2E9F7E0FDC084
:1026B000412F469546954695612F70E0E091540173
:1026C000F0915501002379F0E40FF11D67707070EF
:1026D00081E090E002C0880F991F6A95E2F720819F
:1026E000282B208319C050E0E40FF51F677070702D
:1026F00021E030E002C0220F331F6A95E2F72095F7
:10270000808182238083E0915601F0915701E40F8C
:10271000F51F8081822380838EE593E0BDCF612FFA
:1027200070E0E0915401F0915501002369F063706D
:10273000707081E090E002C0880F991F6A95E2F7FF
:102740002181282B218314C06370707021E030E058
:1027500002C0220F331F6A95E2F720958181822300
:102760008183E0915601F091570181818223818319
:1027700080E793E091CF612F70E0E0915401F091F8
:102780005501002379F0637070706C5F7F4F81E0BA
:1027900090E002C0880F991F6A95E2F72181282BEB
:1027A000218316C0637070706C5F7F4F21E030E052
:1027B00002C0220F331F6A95E2F7209581818223A0
:1027C0008183E0915601F0915701818182238183B9
:1027D00083E893E061CF86E993E061C085ED93E003
:1027E0000E94E41681E0809325078091930780334F
:1027F00009F053C0109225074DC01092A30180E04C
:1028000090E0E0914A01F0914B01E80FF91F10822E
:10281000019688309105A9F70E94F10F46CF1092DA
:10282000A40180E090E0E0915601F0915701E80F9B
:10283000F91F108201968B309105A9F70E941210A2
:1028400034CF81E08093130580919307803309F0A2
:102850002CCF1092130529CF81E080931105809130
:102860009307803309F021CF109211051ECF0E94EB
:10287000680F1BCF0E94701018CF8AEE93E00E9461
:10288000E41681E08093140580919307803329F446
:102890001092140581EE93E002C086EE93E00E9450
:1028A000E41603CF0E94F40D00CF119287E0E23BC3
:1028B000F807D9F710929107109233051F910F91E5
:1028C00008951092B10787EF93E00E94E41682E921
:1028D00097E00E94E41680919207853611F18636C2
:1028E00078F4873479F1883420F4853409F067C0AE
:1028F00015C0803509F446C0843609F060C04BC06D
:10290000883691F0893620F4873609F058C02AC0FD
:102910008037D9F1833709F052C03AC00E944E0285
:102920004EC00E9449024BC085ED93E00E94E41620
:1029300081E080932507809193078033E1F5109221
:10294000250736C01092A50180E090E0E0914A0191
:10295000F0914B01E80FF91F108201968830910524
:10296000A9F72DC01092A50180E090E0E0915601FA
:10297000F0915701E80FF91F108201968B309105F5
:10298000A9F71DC00E94EE0E1AC00E94430E17C088
:102990000E94680F14C08AEE93E00E94E41681E062
:1029A0008093140580919307803329F410921405C5
:1029B00081EE93E002C086EE93E00E94E4168CEF75
:1029C00093E00E94E416E2E9F7E0119287E0E23B2F
:1029D000F807D9F708951DB88091800780FF02C0DD
:1029E0006D9A01C06D988DB180916D0780FF02C016
:1029F0006B9A01C06B988DB180917E0780FF02C0F9
:102A00006A9A01C06A988DB180917F07833091F0F6
:102A1000843028F4813051F0823050F410C0853079
:102A200089F0853048F0863051F407C0699A0AC0B1
:102A3000699A03C0689A06C0689A709A04C08DB1FA
:102A400083608DB970988DB180658DB9089584E0EB
:102A500080937F071092800710926D0710927E0777
:102A60000E94EB14089586E080937F071092800700
:102A700081E080936D0780937E070E94EB14089598
:102A800010927F071092800710926D0710927E07B8
:102A90000E94EB140895873008F086E080937F074A
:102AA0000E94EB140895811181E0809380070E94B9
:102AB000EB140895811181E080936D070E94EB145F
:102AC0000895811181E080937E070E94EB140895A0
:102AD0006C9B6C9A8FB9779BFECF8FB10895AF92A4
:102AE000BF92CF92DF92EF92FF920F931F93CF93FB
:102AF000DF93C82ED62EEE24FF24862F90E027E207
:102B0000A22E25E0B22EA80EB91EEC01CC5FDB4F41
:102B100001E010E07FC0C39AF50180818823C1F0F5
:102B2000DD2059F428B38881A80102C0440F551F45
:102B30008A95E2F7242B28BB26C022B38881F801AE
:102B400002C0EE0FFF1F8A95E2F72E2B22BB1BC09F
:102B5000DD2069F428B38881A80102C0440F551F05
:102B60008A95E2F7CA018095822388BB0CC022B304
:102B70008881F80102C0EE0FFF1F8A95E2F7CF01AE
:102B80008095822382BBC398F701E259F84F808178
:102B90000E946815F701EF57F84F8083C39AF5013B
:102BA00080818823E1F0DD2069F428B38881A801C1
:102BB00002C0440F551F8A95E2F7CA01809582230F
:102BC00088BB24C022B38881F80102C0EE0FFF1F2A
:102BD0008A95E2F7CF018095822382BB17C0DD2062
:102BE00059F428B38881A80102C0440F551F8A9563
:102BF000E2F7242B28BB0AC022B38881F80102C067
:102C0000EE0FFF1F8A95E2F72E2B22BBC398089484
:102C1000E11CF11CEC1408F47ECFDF91CF911F91E1
:102C20000F91FF90EF90DF90CF90BF90AF900895FD
:102C3000FF920F931F93CF93DF93F82E042F44231B
:102C400079F488B39091040421E030E002C0220FAF
:102C5000331F9A95E2F7822788BBEB0110E014C07E
:102C600022B3E42FF0E0EC5FFB4F308181E090E095
:102C700002C0880F991F3A95E2F7282722BBEDCFB3
:102C800089910E9468151F5F1F15D0F3002369F416
:102C900088B39091040421E030E002C0220F331F7A
:102CA0009A95E2F7822788BB0FC022B3E02FF0E0AD
:102CB000EC5FFB4F308181E090E002C0880F991FEC
:102CC0003A95E2F7282722BBDF91CF911F910F9110
:102CD000FF900895982F6C9A20E030E011C0C498BE
:102CE000F901E259F84F80818FB9F901EF57F84F98
:102CF00002C08FB18083779BFCCFC49A2F5F3F4F78
:102D0000291768F3089588E085BD85B5836085BD82
:102D10008CE783BD89B7806889BF08951F920F92A1
:102D20000FB60F9211242F938F939F93AF93BF935E
:102D300080912B0590912C05875E934050F48091F3
:102D40002B0590912C05019690932C0580932B05D3
:102D500017C010922C0510922B0580912D05909193
:102D60002E05A0912F05B09130050196A11DB11D32
:102D700080932D0590932E05A0932F05B0933005D9
:102D8000BF91AF919F918F912F910F900FBE0F9098
:102D90001F90189510BC83E389B91BB81AB8549AD0
:102DA0008898579A539A899A86E880BD08955D9BC2
:102DB000FECF8CB908955D9BFECF8DE08CB95D9BF5
:102DC000FECF8AE08CB90895FC0104C05D9BFECF64
:102DD00031968CB980818823C9F70895FC0104C01D
:102DE0005D9BFECF31968CB980818823C9F7089509
:102DF000FC0104C05D9BFECF31968CB98081882395
:102E0000C9F75D9BFECF8DE08CB95D9BFECF8AE05C
:102E10008CB908950E94E4165D9BFECF8DE08CB9BD
:102E20005D9BFECF8AE08CB908951F920F920FB67A
:102E30000F9211248F939F93EF93FF939CB19093E4
:102E40003605809133058823A9F59D3089F480915A
:102E50003405E82FF0E0EE56F84F1082809391078A
:102E6000109234051092350581E08093330522C01D
:102E7000809135058823F1F49F3511F09B3321F4BF
:102E800081E08093350516C0983031F48091340587
:102E9000882381F081500CC0903260F0809134051D
:102EA0008F3140F4E82FF0E0EE56F84F90838F5FBB
:102EB00080933405FF91EF919F918F910F900FBEFA
:102EC0000F901F9018950E9479090E94E4160895AA
:102ED0000E9412090E94E41608950E94830A0E942B
:102EE000E41608950E94A00B0E94E41608950E9423
:102EF000EC080E94E41608950E94BC0C0E94E4169F
:102F000008950E941F0D0E94E41608950E94D008A3
:102F10000E94E41608950E94BA080E94E4160895DB
:102F20000E947B0D0E94E41608950E94B90D0E9434
:102F3000E4160895EF92FF920F931F937B018C018B
:102F400020E030E040E05FE40E946A1A88238CF0C1
:102F5000C801B70120E030E040E05FE40E941219B0
:102F60000E94531B9B01AC01205030404040504810
:102F700006C0C801B7010E94531B9B01AC01B901F7
:102F8000CA011F910F91FF90EF900895A0E0B0E06B
:102F9000ECECF7E10C946A1EDC012B01FA019C9128
:102FA000923008F439C1EB018881823008F433C1D2
:102FB000943069F4843009F02FC111969C911197D7
:102FC0008981981709F428C1A8E0B4E025C18430AC
:102FD00009F421C18230A9F4923009F01DC19A018F
:102FE000AD0188E0EA010990AE01E90109929E0174
:102FF0008150C1F7E201898111969C9189238183D7
:1030000008C1923009F407C112962D903C90139795
:10301000EB018A819B811496AD90BD90CD90DC90A0
:103020001797EC80FD800E811F819101281B390BC1
:10303000B90137FF04C066277727621B730B603224
:1030400071050CF061C0121613066CF537014801CA
:10305000062E04C096948794779467940A94D2F7C6
:1030600021E030E040E050E004C0220F331F441F55
:10307000551F6A95D2F721503040404050402E21D4
:103080003F2140235123211531054105510521F0F0
:1030900021E030E040E050E079018A01E628F7289D
:1030A000082919293CC0232BD1F1260E371E3501E2
:1030B0004601062E04C096948794779467940A94E8
:1030C000D2F721E030E040E050E004C0220F331F8F
:1030D000441F551F6A95D2F7215030404040504060
:1030E0002A213B214C215D21211531054105510546
:1030F00021F021E030E040E050E059016A01A628CB
:10310000B728C828D9280BC0821593052CF01C01BC
:10311000AA24BB24650103C0EE24FF248701119675
:103120009C91D20111968C91981709F445C099236E
:1031300039F0A80197012A193B094C095D0906C01D
:10314000A60195012E193F09400B510B57FD08C0F0
:1031500011823382228224833583468357831DC0A4
:1031600081E081833382228288279927DC01821BB8
:10317000930BA40BB50B84839583A683B7830DC0F3
:10318000220F331F441F551F2483358346835783E3
:103190008281938101979383828324813581468143
:1031A0005781DA01C9010197A109B1098F5F9F4FCA
:1031B000AF4FBF4328F30BC0918333822282EA0CC6
:1031C000FB1C0C1D1D1DE482F5820683178383E022
:1031D0008083248135814681578157FF1AC0C901F8
:1031E000AA2797FDA095BA2F81709070A070B0703B
:1031F0005695479537952795822B932BA42BB52B66
:1032000084839583A683B783828193810196938378
:103210008283DF0101C0D201CD01CDB7DEB7E2E18B
:103220000C94861EA0E2B0E0E8E1F9E10C94761E71
:1032300069837A838B839C832D833E834F83588756
:10324000E9E0EE2EF12CEC0EFD1ECE010196B70149
:103250000E94441D8E010F5E1F4FCE010596B801DE
:103260000E94441D8A8991E089278A8BC701B80191
:10327000AE01475E5F4F0E94C6170E946F1CA0966A
:10328000E6E00C94921EA0E2B0E0E9E4F9E10C94CF
:10329000761E69837A838B839C832D833E834F8341
:1032A0005887F9E0EF2EF12CEC0EFD1ECE010196B1
:1032B000B7010E94441D8E010F5E1F4FCE0105967F
:1032C000B8010E94441DC701B801AE01475E5F4FBF
:1032D0000E94C6170E946F1CA096E6E00C94921EF6
:1032E000A0E2B0E0E6E7F9E10C946A1E69837A8314
:1032F0008B839C832D833E834F835887CE01019619
:10330000BE01675F7F4F0E94441DCE010596BE013E
:103310006F5E7F4F0E94441D9985923088F08989A5
:103320008230C8F0943019F4823051F404C08430F3
:1033300029F4923081F488E094E0C6C0923049F4D8
:1033400020E09A858A89981321E02A87CE01099680
:10335000BBC0823049F420E09A858A89981321E025
:103360002A8BCE014196B0C02D843E844F8458886C
:103370006D887E888F88988CEE24FF248701AA248C
:10338000BB24650140E050E060E070E0E0E0F0E088
:10339000C10181709070892BE9F0E60CF71C081DC3
:1033A000191D9A01AB012A0D3B1D4C1D5D1D80E0CE
:1033B00090E0A0E0B0E0E614F7040805190520F459
:1033C00081E090E0A0E0B0E0BA01A901480F591FE8
:1033D0006A1F7B1FAA0CBB1CCC1CDD1C97FE08C0FF
:1033E00081E090E0A0E0B0E0A82AB92ACA2ADB2A4E
:1033F0003196E032F10549F0660C771C881C991C67
:103400005694479437942794C3CFFA85EA892B8939
:103410003C898B859C85280F391F2E5F3F4F17C035
:10342000CA0181709070892B61F016950795F79409
:10343000E79480E090E0A0E0B0E8E82AF92A0A2BBF
:103440001B2B76956795579547952F5F3F4F77FDD7
:10345000E7CF0CC0440F551F661F771F17FD416053
:10346000EE0CFF1C001F111F21503040403090E037
:10347000590790E0690790E4790760F32B8F3C8F40
:10348000DB01CA018F779070A070B0708034910515
:10349000A105B10561F447FD0AC0E114F10401057D
:1034A000110529F0405C5F4F6F4F7F4F40781A8EB7
:1034B000FE1711F081E08A8F4D8F5E8F6F8F78A39A
:1034C00083E0898FCE0149960E946F1CA096E2E1AD
:1034D0000C94861EA8E1B0E0E0E7FAE10C94761EB9
:1034E00069837A838B839C832D833E834F835887A4
:1034F00089E0E82EF12CEC0EFD1ECE010196B701FD
:103500000E94441D8E010F5E1F4FCE010596B8012B
:103510000E94441D8985823040F08989823028F0DC
:10352000C701B8010E94BC1D01C08FEF6896E6E09C
:103530000C94921EA8E1B0E0E0EAFAE10C94761E49
:1035400069837A838B839C832D833E834F83588743
:1035500089E0E82EF12CEC0EFD1ECE010196B7019C
:103560000E94441D8E010F5E1F4FCE010596B801CB
:103570000E94441D8985823040F08989823028F07C
:10358000C701B8010E94BC1D01C081E06896E6E059
:103590000C94921EA8E1B0E0E0EDFAE10C947A1EE2
:1035A00069837A838B839C832D833E834F835887E3
:1035B000CE010196BE01675F7F4F0E94441DCE0180
:1035C0000596BE016F5E7F4F0E94441D8985823043
:1035D00028F020E030E08989823010F421E030E0EA
:1035E000822F6896E2E00C94961EA8E0B0E0EBEF24
:1035F000FAE10C94731E9B01AC0183E08983DA012C
:10360000C9018827B7FD83959927AA27BB27B82E1C
:10361000211531054105510519F482E089833AC02D
:103620008823A9F0203080E0380780E0480780E850
:10363000580729F460E070E080E09FEC30C0EE2491
:10364000FF248701E21AF30A040B150B02C079016B
:103650008A018EE1C82ED12CDC82CB82ED82FE82E3
:103660000F831887C801B7010E94201C0197181604
:10367000190684F4082E04C0EE0CFF1C001F111F55
:103680000A94D2F7ED82FE820F831887C81AD90AEE
:10369000DC82CB82BA82CE0101960E946F1C2896F2
:1036A000E9E00C948F1EACE0B0E0E9E5FBE10C949E
:1036B0007A1E69837A838B839C83CE010196BE0137
:1036C0006B5F7F4F0E94441D8D81823061F182309B
:1036D00050F1843021F48E81882351F12EC02F8146
:1036E000388537FD20C06E812F3131051CF06623EF
:1036F000F9F023C08EE190E0821B930B29853A8577
:103700004B855C8504C056954795379527958A95D6
:10371000D2F76623B1F050954095309521953F4FF3
:103720004F4F5F4F0EC020E030E040E050E009C056
:103730002FEF3FEF4FEF5FE704C020E030E040E0C5
:1037400050E8B901CA012C96E2E00C94961EA8E05C
:10375000B0E0EDEAFBE10C94721E7B018C01611577
:1037600071058105910519F482E0898360C083E0C9
:1037700089838EE1C82ED12CDC82CB82ED82FE8241
:103780000F831887C801B7010E94201CFC013197E4
:10379000F7FF3BC0222733272E1B3F0B5701680141
:1037A000022E04C0D694C794B794A7940A94D2F773
:1037B00040E050E060E070E081E090E0A0E0B0E048
:1037C00004C0880F991FAA1FBB1F2A95D2F7019723
:1037D000A109B1098E219F21A023B1230097A10542
:1037E000B10521F041E050E060E070E04A295B293A
:1037F0006C297D294D835E836F8378878EE190E00D
:103800008E1B9F0B9C838B8312C0309781F00E2EF2
:1038100004C0EE0CFF1C001F111F0A94D2F7ED82AA
:10382000FE820F831887CE1ADF0ADC82CB821A82CF
:10383000CE0101960E946F1C2896EAE00C948E1E21
:10384000EF92FF920F931F937B018C0180E0E816AB
:1038500080E0F80681E0080780E0180788F48FEF21
:10386000E816F1040105110531F028F088E090E038
:10387000A0E0B0E017C080E090E0A0E0B0E012C0AF
:1038800080E0E81680E0F80680E0080781E018078D
:1038900028F088E190E0A0E0B0E004C080E190E092
:1038A000A0E0B0E020E230E040E050E0281B390B1F
:1038B0004A0B5B0B04C016950795F794E7948A951D
:1038C000D2F7F701E05FFB4F8081281B31094109E6
:1038D0005109C9011F910F91FF90EF900895DF9258
:1038E000EF92FF920F931F93FC01E480F580068115
:1038F0001781D1808081823048F480E090E0A0E19F
:10390000B0E0E82AF92A0A2B1B2BA5C0843009F461
:103910009FC0823021F4EE24FF24870105C0E1140A
:10392000F1040105110519F4E0E0F0E096C06281B0
:1039300073819FEF623879070CF05BC022E83FEF9C
:10394000261B370B2A3131052CF020E030E040E017
:1039500050E02AC0B801A701022E04C076956795F1
:10396000579547950A94D2F781E090E0A0E0B0E047
:1039700004C0880F991FAA1FBB1F2A95D2F7019771
:10398000A109B1098E219F21A023B1230097A10590
:10399000B10521F081E090E0A0E0B0E09A01AB0138
:1039A000282B392B4A2B5B2BDA01C9018F779070BA
:1039B000A070B07080349105A105B10539F427FFDE
:1039C00009C0205C3F4F4F4F5F4F04C0215C3F4F09
:1039D0004F4F5F4FE0E0F0E02030A0E03A07A0E07A
:1039E0004A07A0E45A0710F0E1E0F0E079018A010B
:1039F00027C06038710564F5FB01E158FF4FD8011D
:103A0000C7018F779070A070B07080349105A105C8
:103A1000B10539F4E7FE0DC080E490E0A0E0B0E02D
:103A200004C08FE390E0A0E0B0E0E80EF91E0A1FAA
:103A30001B1F17FF05C016950795F794E79431965D
:103A400087E016950795F794E7948A95D1F705C016
:103A5000EE24FF248701EFEFF0E06E2F67956627D5
:103A60006795902F9F77D794DD24D7948E2F8695D6
:103A7000492F462B582F5D29B701CA011F910F917D
:103A8000FF90EF90DF900895FC01DB0140815181B0
:103A90002281622F6F7770E0221F2227221F9381DD
:103AA000892F880F822B282F30E0991F9927991F83
:103AB00011969C93119721153105A9F541155105D2
:103AC0006105710511F482E037C082E89FEF13961B
:103AD0009C938E9312979A01AB0167E0220F331FDC
:103AE000441F551F6A95D1F783E08C930DC0220FB8
:103AF000331F441F551F12968D919C911397019768
:103B000013969C938E931297203080E0380780E0C4
:103B1000480780E4580758F314962D933D934D932E
:103B20005C93179708952F3F310579F4411551059E
:103B30006105710519F484E08C93089564FF03C056
:103B400081E08C9312C01C9210C02F573040139606
:103B50003C932E93129783E08C9387E0440F551F7C
:103B6000661F771F8A95D1F7706414964D935D9305
:103B70006D937C93179708951F93DC01FB019C9133
:103B8000923008F447C08081823008F443C09430FA
:103B900051F411961C91843099F58181682F70E061
:103BA000611B71093FC0843021F0923031F48230C2
:103BB000B9F18181882389F12DC011961C9111974B
:103BC0008230F1F081811817D9F412962D913C9131
:103BD0001397828193818217930794F028173907EE
:103BE000BCF014968D919D910D90BC91A02D2481D7
:103BF000358146815781281739074A075B0718F432
:103C0000112341F00AC082179307A407B50740F4B7
:103C1000112319F061E070E005C06FEF7FEF02C083
:103C200060E070E0CB011F910895991B79E004C01A
:103C3000991F961708F0961B881F7A95C9F78095EB
:103C40000895AA1BBB1B51E107C0AA1FBB1FA617E3
:103C5000B70710F0A61BB70B881F991F5A95A9F735
:103C600080959095BC01CD01089597FB092E0726FC
:103C70000AD077FD04D0E5DF06D000201AF4709555
:103C800061957F4F0895F6F7909581959F4F089520
:103C9000A1E21A2EAA1BBB1BFD010DC0AA1FBB1F50
:103CA000EE1FFF1FA217B307E407F50720F0A21BC2
:103CB000B30BE40BF50B661F771F881F991F1A942F
:103CC00069F760957095809590959B01AC01BD0159
:103CD000CF0108952F923F924F925F926F927F9201
:103CE0008F929F92AF92BF92CF92DF92EF92FF920C
:103CF0000F931F93CF93DF93CDB7DEB7CA1BDB0BB8
:103D00000FB6F894DEBF0FBECDBF09942A8839885C
:103D100048885F846E847D848C849B84AA84B98463
:103D2000C884DF80EE80FD800C811B81AA81B9816F
:103D3000CE0FD11D0FB6F894DEBF0FBECDBFED0183
:063D40000895F894FFCF86
:103D460073657474696E67206F662041546D65678C
:103D56006120696E7465726E616C20414443206512
:103D66006E61626C65207265676973746572732033
:103D76006973206E6F7420737570706F72746564EA
:103D86002E207965742E0A000A2073657420656EEC
:103D960061626C652062697473206F6620414437E6
:103DA60037313920506F7274200020746F20002044
:103DB600746F20307846460A0020746F20307830C1
:103DC600300A000A20736F6D657468696E67207724
:103DD600726F6E670A0075736172745F72785F62E4
:103DE60075666665725F696E6465783A20000A20BA
:103DF60075736172745F72785F6275666665725B11
:103E0600325D3A20000A2075736172745F72785FC2
:103E16006275666665725B345D3A200038053C055E
:103E26003E05400542057C055605690546054705DC
:103E360048057C065E0571054C054D054E0563611A
:103E4600726574616B657221206572726F72206390
:103E56006F64653A00657468676F743A00567C0053
:103E660050432073656E64696E6720746F206661C7
:103E76007374210A0063683A0020763A002073754D
:103E86006D3A0001010146534320302E32200A20AC
:103E96006275696C643A2030352E30362E323031F8
:103EA600300A006C72703A006F66663A007361649D
:103EB6003A006E72703A0048696C666565656565BC
:103EC600656565656565656565650A00013031325C
:103ED60033343536373839414243444546007072EB
:103EE600696E74696E672068656C703A202D6E6F16
:103EF60074207965742D200A000A207072696E7428
:103F0600696E6720766F6C746167657320696E20D1
:103F16006D563A0A00202020007072696E74696E30
:103F26006720766F6C746167657320696E206D56C5
:103F3600202D20737475706964206D6F64653A0A6C
:103F46000063683A00523A000A207072696E74691A
:103F56006E67206D6561737572656420726573693D
:103F66007374616E636520696E206B6F686D733A5A
:103F76000A002000202020202020200061646320E9
:103F86007374617475733A0A006164373731392086
:103F96007374617475733A0A0074696D653A00202A
:103FA6007365632E0A0054657374204168204121AD
:103FB600210A007374617475733A200074696D6523
:103FC6005F733A20002E00564F4C54414745530A22
:103FD60000656E61626C653A002020646F6E653A1A
:103FE6000076616C7565733A0052455349535441E6
:103FF6004E4345530A0076616C7565733A0A000AAA
:10400600656E642E0A00706172736765743A000A01
:1040160020492077696C6C20737769746368200087
:104026006F6E20006F666620002072657369737478
:10403600616E6365206368616E6E656C2000207634
:104046006F6C74616765206368616E6E656C2000D5
:104056002068756D6964697479206368616E6E6540
:104066006C200020707265737375726520636861D9
:104076006E6E656C20000A2044414D4E2120746806
:1040860069732073686F756C64206E65766572203F
:1040960068617070656E2D20656E61626C652F6457
:1040A600697361626C65207377697463682D6361F7
:1040B6007365210A000A686561727462656174201D
:1040C600006F66660A006F6E0A000A6465627567AD
:1040D600206D6F64652000676F743A000A7265612F
:1040E60064793F000403040500000000000000009E
:1040F6000001020203030303040404040404040489
:104106000505050505050505050505050505050559
:104116000606060606060606060606060606060639
:104126000606060606060606060606060606060629
:104136000707070707070707070707070707070709
:1041460007070707070707070707070707070707F9
:1041560007070707070707070707070707070707E9
:1041660007070707070707070707070707070707D9
:1041760008080808080808080808080808080808B9
:1041860008080808080808080808080808080808A9
:104196000808080808080808080808080808080899
:1041A6000808080808080808080808080808080889
:1041B6000808080808080808080808080808080879
:1041C6000808080808080808080808080808080869
:1041D6000808080808080808080808080808080859
:1041E6000808080808080808080808080808080849
:00000001FF
